:020000040000FA
:040000001EEF01F0FE
:060008000001B7D8110051
:10001800D8CF00F0E0CF01F0026EE9CF03F0EACFCD
:1000280004F09DA827D09EA825D09D9841BC05D056
:100038002AAE03D0418227801DD081A01BD0066A3A
:1000480041BC0AD0B06A2F0E056E81B003D0010EF4
:10005800066E02D0052EF9D706660AD001EE40F0EA
:100068003B50E926EFCFADFF418C3B2A320602D048
:10007800418227809DAA47D09EAA45D04A6A076A2E
:10008800ABA203D0AB98AB8832D0ABA409D0AE50AA
:10009800010E076E41A02BD04A0EAF6E419027D0BB
:1000A800AECF05F005BE356A01EE00F03550E92601
:1000B80005C0EFFF41A004D04A0EAF6E419012D0A8
:1000C80041AC10D001EE40F03A50E926EFCF06F0EF
:1000D8000550061803E0010E076E04D03A2A3A9A32
:1000E80032669D88076603D02782352A359A41AC47
:1000F8000AD0075208E0419C9D98418227807C0ED7
:10010800AF6EAD6A41809EA22AD09E922E5221E007
:10011800076A09EED8F0080E056E2EAE04D0EF502F
:10012800066201D0078E07462E46EE50052EF5D7FB
:1001380007520FE007502D1A2E1A2DC081FF2DA04F
:10014800829A2DB0828A8B988B882E6602D0066898
:10015800CA94062A3A0E066402D0066ACA9403C0F4
:10016800E9FF04C0EAFF025001C0E0FF00C0D8FF69
:100178001000F2A812D0F2A210D0F292F2980A0E51
:10018800BA6F586A2A8E4A6A27B007D041BC05D090
:100198000D0E3E6002D0020E3E26120063BE09D04C
:1001A800D6CF08F06650085C675E08C066F0D8A035
:1001B800638E1200D6CF08F06450085C655E08C0F4
:1001C80064F0D8B012009C0E6526400E6826D8B0A0
:1001D800652A050E096E010E0A6E00EE59F063508D
:1001E8000A140DE1EF06EF3C03D0EE50EF06ED5098
:1001F800EF50EE50EF1002E10A506312ED50020E7C
:10020800E926000EEA22D8900A36092EE8D712000D
:100218000B6E0C6A100E0D6E09360A360C360E3649
:100228000B500C5C0EB0D880D8B00C6E0D2EF4D7E5
:100238000C501200B7EC19F0EFEC19F0000115ECB6
:100248001AF0000159EC1AF06368646A656AC40E12
:10025800D56E276A27862788278AD08EF28EF28C59
:10026800446A456A466A476A800E576E586E486AFD
:10027800496A4A6E4B6A4C6E4D6A4E6A4F6A506EB6
:10028800516E526E536E546E556E566E0400D19078
:10029800000184DF8FDF44BE03D017EC06F0446E04
:1002A80045BE03D0A0EC06F0456E46BE03D0E3EC95
:1002B80006F0466E47BE05D0010124EC07F0476EF4
:1002C800000148BE04D0010189D8486E000149BE2A
:1002D80004D001011BD9496E00014ABE02D042D8A0
:1002E8004A6E4BBE02D0A2D84B6E4CBE02D032D959
:1002F8004C6E4DBE02D049D94D6E4EBE02D095D936
:100308004E6E4FBE02D049DA4F6E50BE03D083EC1A
:1003180007F0506E51BE02D072DB516E52BE03D050
:100328008DEC05F0526E53BE03D053EC11F0536EB2
:1003380054BE03D0A4EC15F0546E55BE03D098EC0F
:1003480017F0556E56BE03D005EC12F0566E57BE28
:1003580003D0BBEC08F0576E58BE9BD7C8EC08F02A
:10036800586E97D7F9504A44F92602D007D032D0B0
:100378002A8ED6CF66F0BB0E676E639E63AE010C05
:10038800F292F2883E44086EF9500844F926BB0EF2
:100398001DD0B20E1BD0A80E19D09F0E17D0960EE6
:1003A80015D08C0E13D0830E11D0790E0FD0700E8D
:1003B8000DD0670E0BD05D0E09D0540E07D04B0E32
:1003C80005D0410E03D0380E01D0000ED6CF66F00E
:1003D800676E639E63AE020C2A9E800CF9504844F7
:1003E800F92600D027A2010C00AF1CD08CEC08F035
:1003F800086E085017E0FF0A03E1006B419C12D019
:1004080011EE00F002EE00F03350E926E6CFEEFFE1
:10041800E950D8B402EE00F0082EF8D7E9CF33F04F
:10042800419C27802792000C0101800C4B50D8A4D6
:10043800800C3350341869E002EE00F03450E9269D
:10044800EFAE62D002EE00F0E926EF50830A0DE02D
:10045800330A10E0010A24E0030A32E05F0A40E0B0
:10046800020A4BE05B0A4EE04FD006017AEC0DF031
:1004780000014AD05DEC18F008C030F009C031F036
:1004880030503114FF0A40E0000E5CEC0CF00EC056
:1004980008F00FC009F05BEC0BF02A94536A34D0D3
:1004A8005DEC18F008C030F009C031F0305031145C
:1004B800FF0A2AE0010E5CEC0CF02A94536A24D05F
:1004C8005DEC18F008C030F009C031F0305031143C
:1004D800FF0A1AE0020E5CEC0CF02A94536A14D05E
:1004E800FEEC17F008C030F009C031F0305031147C
:1004F800FF0A0AE02A84536A07D00601FCEC0DF0D3
:10050800000102D01FEC11F0342A000CF9504944C4
:10051800F92603D002D00DD012D027A4010C2794BD
:1005280040390F0B3E6E0F0E4015326E010E3A6EBB
:100538003B6E2ABE01D041AA020C9D88279027A0B5
:10054800030C41A202D04192EED73E6A2786000CE6
:100558000101800CF9504C44F92600D027A6010C63
:10056800279611EE20F0E6CF08F021EE40F008C003
:10057800DEFF0806096AE6CFDFFFDE50091A082EFB
:10058800FAD7091CDF6E2784800CF9504D44F926F0
:1005980001D006D03850366203D03950371844E0BD
:1005A80027A6010C279621EE40F03650E96E030E7F
:1005B8003724EA6EEFCF08F008C0DEFF362A000EB7
:1005C8003722366605D0020E376202D0366A376A9D
:1005D8000806096A3650E96E030E3724EA6EEFCF33
:1005E800DFFFDE50091A362A000E3722366605D09C
:1005F800020E376202D0366A376A082EEBD7091C1A
:10060800DF6E3650385C086E37503958096E09AEBF
:1006180002D0020E092609BE05D0D00E085C010ED4
:100628000958D8A027882784000CF9504E44F92689
:1006380002D00CD013D08C53D8B4AED06A68010E57
:10064800696E6952D8B4A5D06A2A010C69508C1514
:10065800D8B49CD0691C8C1741A427D027A8020CB9
:10066800080E6A02F350990FD96E090EDA6ADA2277
:10067800DDCF0CF00CBC8AD00C38030BD8A486D084
:10068800DECF0DF00E6ADFCF0EF0695086150E88AA
:10069800D8B40E98100E206E24900DC021F00EC014
:1006A80022F06A50D4EC0AF071D0080E6A02F350B6
:1006B800990FD96E090EDA6ADA22DECF08F0DECF9A
:1006C80009F0DECF0AF00F0E0A140B6E0A38070B7A
:1006D8000A6E0A5006E0010A04E0030A02E0010A71
:1006E80055E10AC00CF00BC00DF008C00EF06AC04E
:1006F8000FF0106A6950FEEC09F00A5203E0020E8E
:100708000A6205D00B5203E0695083153FE0D89088
:100718000932D8900932DCBE19D0030E0914010A37
:1007280005E0030A09E0010A0FE010D069508315BB
:100738000DE06950B4130AD06950831507E108BE6B
:1007480005D06950B41302D06950B413D890093257
:10075800D8900932DE50DCBE19D0030E0914010A04
:1007680005E0030A09E0010A0FE010D0695083157B
:100778000DE06950B7130AD06950831507E108BE28
:1007880005D06950B71302D06950B713D8906936AD
:1007980058D7835143EC11F0000CF9504F44F92617
:1007A80002D019D026D08D6703D08E53D8B426D165
:1007B800010E6B6E030E6B6021D16D68010E6C6EBD
:1007C8006C52D8B419D16D2A020E6B6203D0060E92
:1007D8006D600FD1010CEA6A8C0E6B24E96E6C50C7
:1007E800EF14D8B406D1EA6A8C0E6B24E96E6C1C3F
:1007F800EF1627A8020C6B2C09D0080E6D02F350D7
:10080800280FD96E060EDA6ADA2208D0080E6D02B1
:10081800F350680FD96E060EDA6ADA22DECF08F0D6
:10082800096ADFCF09F0DECF0AF0DECF0BF0DECFAA
:100838000CF0EA6A860E6B24E96E6C50EF14098896
:10084800D8B409980A38030B03E141A462D0D1D087
:100858000C38070B5EE141B45CD0EA6A800E6B2469
:10086800E96E6C50EF1416E0EA6A800E6B24E96EAC
:100878006C1CEF16EA6AAB0E6B24E96E6C50EF1431
:10088800D880D8B4D89003E209B8B3D042D009B818
:1008980040D0AFD0EA6AB10E6B24E96E6C50EF1409
:1008A80022E1EA6AAB0E6B24E96E6C1CEF1609A80C
:1008B80010D06C50EF12030E0B14030A2AE00CC080
:1008C8000DF06DC00EF06BC00FF06C509EEC0AF08E
:1008D80090D00CC00DF06DC00EF06BC00FF06C50D6
:1008E8009EEC0AF086D0EA6AAB0E6B24E96E6C5077
:1008F800EF14D880D8B4D89003E209B803D009D04F
:1009080009B807D0EA6AB10E6B24E96E6C1CEF16C1
:1009180070D0030E0B14010A07E0030A08E0010A6D
:1009280008E0030A30E005D009B803D02CD009B894
:100938002AD00A38030B1DE1EA6A890E6B24E96E96
:10094800EFCF0DF009BE03D06C500D1A07D06DA083
:1009580003D06C500D1202D06C1C0D166C500D1487
:100968000988D8B40998EA6A890E6B24E96E0DC023
:10097800EFFF0AC020F0249008C021F009C022F03F
:100988006D50D4EC0AF041B434D0D8900B32D890E2
:100998000B32030E0B14010A07E0030A08E0010AF0
:1009A80008E0030A0CE005D009B803D008D009B85C
:1009B80006D0EA6AB40E6B24E96E6C50EF12D89038
:1009C8000B32D8900B32030E0B14010A07E0030A0E
:1009D80008E0010A08E0030A0CE005D009B803D0D2
:1009E80008D009B806D0EA6AB70E6B24E96E6C50D5
:1009F800EF12D8906C36E4D66B2ADCD6000CF9508E
:100A08005144F92602D018D02BD06E6A030E6E60BE
:100A18007FD0EA6AB40E6E24E96EEF5077E0706812
:100A2800010E6F6E6F5272E0702A020E6E6203D072
:100A3800060E706068D0010CEA6A8C0E6E24E96EAE
:100A48006F50EF1460E1EA6AB40E6E24E96E6F50DD
:100A5800EF1459E0EA6AB40E6E24E96E6F1CEF16C3
:100A680027A8020C6E6609D0080E7002F350980F82
:100A7800D96E090EDA6ADA2213D06E2C09D0080E64
:100A88007002F350280FD96E060EDA6ADA2208D0FF
:100A9800080E7002F350680FD96E060EDA6ADA2271
:100AA800DCCF08F0030ED926000EDA22DECF09F0DB
:100AB8000A6ADFCF0AF0DFCF0BF0EA6A860E6E24EF
:100AC800E96E6F50EF140A88D8B40A980C9008BEE3
:100AD8000C806E520EE00CB00CD00838030B09E104
:100AE800EA6A890E6E24E96E6F50EF140A88D8B44A
:100AF8000A980BC020F0248009C021F00AC022F017
:100B08007050D4EC0AF0D8906F368CD76E2A7ED706
:100B1800800CF9505244F92602D018D025D0716AB9
:100B2800030E71607FD0EA6AB70E7124E96EEF5048
:100B380077E07368010E726E725272E0732A020EC9
:100B4800716203D0060E736068D0010CEA6A8C0EDD
:100B58007124E96E7250EF1460E1EA6AB70E7124ED
:100B6800E96E7250EF1459E027A8020CEA6AB70E32
:100B78007124E96E721CEF16716609D0080E7302B3
:100B8800F350980FD96E090EDA6ADA2213D0712C55
:100B980009D0080E7302F350280FD96E060EDA6AD0
:100BA800DA2208D0080E7302F350680FD96E060EC9
:100BB800DA6ADA22DCCF08F0050ED926000EDA222E
:100BC800DECF09F00A6ADFCF0AF0DFCF0BF0EA6A5E
:100BD800860E7124E96E7250EF140A88D8B40A9808
:100BE8000C9008BE0C8071520EE00CB00CD0083886
:100BF800030B09E1EA6A890E7124E96E7250EF1459
:100C08000A88D8B40A980BC020F0248009C021F0C3
:100C18000AC022F07350D4EC0AF0D89072368CD700
:100C2800712A7ED7800CF9504444F92602D005D0A9
:100C380025D0010E596E5A6A639063A0010C2AA64A
:100C4800E7EC14F0742A400E746404D0010E746E3C
:100C580056EC14F0070E7414D8B41BEC14F0752A73
:100C6800060E7560756A050E756203D0230EC26E96
:100C780005D0040E7502F350030FC26EC2B2020C07
:100C8800010E086E755005E00D6ED89008360D2ED1
:100C9800FCD788C00AF0B0510A1AC4CF0CF0C3CFF1
:100CA8000BF0BD0E0B5C020E0C580EE308500A1434
:100CB8000BE108500A12B0510A1A0AC088F041AA7A
:100CC80015D008508E1312D05E0E0B5C010E0C5816
:100CD8000DE208500A140AE0081C0A16B0510A1A54
:100CE8000AC088F041AA02D008508E13756623D036
:100CF8002AB63CEC15F087C009F02CEC11F00B6E0D
:100D08000BC084F009180C6E010E086E08520AE038
:100D180076500C14081403E00850871B8D13D890E4
:100D28000836F4D70CC076F02AA805D0BC2F03D01B
:100D38002A98948A278A000CF9504544F92601D04C
:100D480004D00A0E5B6E5C6A639263A2010C506A5F
:100D5800556A566A516A526A81B008D041AA0DD0C4
:100D68003C2A0A0E3C6209D0419A07D03C6A41BA33
:100D780004D03D6602D0010E3D6E3D520FE03D2A83
:100D8800180E3D640BD03D6AF29EF292F288AB8851
:100D98009E9A9D8A9D98AC8AF28E418A41A40ED073
:100DA800086A030E086007D0EA6A8C0E0824E96E08
:100DB800EF10082AF6D7FF0AD8A44194000CF9507E
:100DC8004644F92601D004D0640E5D6E5E6A6394D1
:100DD80063A4010CBD530EE0BD070F0EBD150AE15B
:100DE800BD3BBD070F0EBD1504E00A0EBB6F576A69
:100DF800BD8BBD3BBE5307E0BE2F05D0500EBB6F69
:100E0800576A0A0EBE6F84B619D0282A41B807D08F
:100E18000A0E28620BD04188010EBE6F07D0020E61
:100E2800286204D04198BE6B650E286E640E286255
:100E380003D0D19000EF00F0000101D0286A000C27
:100E48000001F9504744F92603D00BD01DD02ED00D
:100E5800E80E5F6E030E606E6396010163B603D001
:100E6800010C0101FBD72AA02DD060C11CF061C183
:100E78001DF0000186515BEC19F0640E616E626A28
:100E8800639863B803D0020C0101FBD760291C6E7C
:100E9800000E61211D6E00018A515BEC19F0640E91
:100EA800616E626A639863B803D0030C0101FBD7D3
:100EB800020E60251C6E000E61211D6E00018B5113
:100EC8005BEC19F041A618D03F5207E04184EA6A6A
:100ED8008C0E3F24E96EEF6809D0060107A906D0F9
:100EE8004184EA6A8C0E3F24E96EEF683F2A020EBD
:100EF80001013F6401D04196000C0101800CF950BA
:100F08005044F92601D01AD0776A030E7760FFD0D3
:100F1800EA6AB10E7724E96EEF50D8B4F6D07A9029
:100F28007968010E786E7852D8B4E6D0792A020E24
:100F3800776203D0060E7960DCD0010CEA6AB10E44
:100F48007724E96E7850EF14D8B4D3D0776609D0F7
:100F5800080E7902F350980FD96E090EDA6ADA2270
:100F680013D0772C09D0080E7902F350280FD96EC8
:100F7800060EDA6ADA2208D0080E7902F350680FF2
:100F8800D96E060EDA6ADA22DCCF08F0DCCF0AF076
:100F9800DCCF09F00938070B0B6E01EE64F0080E80
:100FA8007702F3507924D890E834E926EE06000E4B
:100FB800EF5A01EE64F0080E7702F3507924D890C6
:100FC800E834E926EE50EF10D8A493D077667FD0A6
:100FD80008AC1AD0080ED926000EDA220938F00B10
:100FE800096E0F0EDF140926080ED95E000EDA5AB4
:100FF8000BC00CF009C00DF079C00EF077C00FF0EF
:10100800785068D97A8075D00B50020A03E0030E35
:101018000B620FD0781CB1170BC00CF00F0E09141F
:101028000D6E0E6A79C00FF0106A7850E3D97A8095
:1010380009D00B5202E00B2C05D0781CB117781C94
:1010480083177A8041B455D0020ED926000EDA22D1
:10105800D8900A32D8900A32DFBE17D0030E0A148D
:10106800010A05E0030A09E0010A0DE00ED07850F4
:1010780083150BE07850B41308D07850831505E138
:101088007850B41302D07850B413020ED926000E4B
:10109800DA22D8900A32D8900A32DFBE2AD0030E5C
:1010A8000A14010A05E0030A09E0010A0DE021D04B
:1010B800785083151EE07850B7131BD078508315ED
:1010C80018E17850B71315D07850B71312D0EA6AE0
:1010D800B10E7724E96E781CEF16EA6A800E772441
:1010E800E96E7850EF12EA6A8C0E7724E96E785030
:1010F800EF12D890783617D77AA007D0EA6A830E0D
:101108007724E96EEF5043EC11F0772AFED6800C75
:1011180000AD11D000AB0CD0010E3564000C01C13C
:1011280009F0030E096403D0100E09640BD0FF0CFC
:10113800060E096E07D000AB03D0040E096E02D06C
:10114800020E096E3550096211D00A6A0B6A01EE67
:1011580000F00B50E926EF500A1A0B2A09500B5CD5
:10116800F6E30A3C02D009501200FF0C000CF950BB
:101178005744F92600D027AA010C279ABBC0BCF017
:101188002A888B8A949A800CF9505844F92600D002
:1011980027AA010C279ABAC0BCF02A888B9A949A7D
:1011A800800C176E010EEA6E16C0E9FF1746174647
:1011B8001744060FF924D8B0FA2AF96EEF6A000E20
:1011C80000003BD00A0EEF6E000E37D0140EEF6E03
:1011D800000E33D0230EEF6E000E2FD0320EEF6EBE
:1011E800000E2BD0410EEF6E000E27D0500EEF6E82
:1011F800000E23D0640EEF6E000E1FD07D0EEF6E32
:10120800000E1BD0960EEF6E000E17D0C80EEF6EB4
:10121800000E13D02C0EEF6E010E0FD0900EEF6E55
:10122800010E0BD0F40EEF6E010E07D0580EEF6EC4
:10123800020E03D0200EEF6E030EEC6E1200176E36
:10124800010EEA6E16C0E9FF17461746F950174413
:10125800F926E80EEF6E030E3BD0DC0EEF6E050E9E
:1012680037D0D00EEF6E070E33D0B80EEF6E0B0EE0
:101278002FD0A00EEF6E0F0E2BD0880EEF6E130E30
:1012880027D0700EEF6E170E23D0280EEF6E230EA8
:101298001FD0E00EEF6E2E0E1BD0500EEF6E460ED6
:1012A80017D0C00EEF6E5D0E13D0300EEF6E750EB8
:1012B8000FD0A00EEF6E8C0E0BD0100EEF6EA40E9A
:1012C80007D0800EEF6EBB0E03D0600EEF6EEA0EF5
:1012D800EC6E1200106EEA6A830E0F24E96EEFCFEF
:1012E80012F00E5005E0156ED8901232152EFCD76C
:1012F800030E12160D14126214D020900DB4208023
:10130800830E0F241E6E105040EC19F020900DB67D
:101318002080830E0F241E6ED890103440EC19F0F4
:1013280013D020900DB02080830E0F241E6E105015
:1013380040EC19F020900DB22080830E0F241E6E11
:10134800D890103440EC19F0EA6A830E0F24E96E45
:10135800EF5043EC11F00D380F0B0D6E080E0F0215
:10136800F3500E24116EEA6AB10E0F24E96E101CB8
:10137800EF160C50020A03E0010A1AE031D0D890A7
:101388001134640F166E0D500CDF01EE64F0D89026
:101398001134E926EECF13F0EECF14F013501410E9
:1013A8001FE0EA6AB10E0F24E96E1050EF1218D050
:1013B800D8901134640F166E0D5041DF01EE64F0C1
:1013C800D8901134E926EECF13F0EECF14F0135075
:1013D800141006E0EA6AB10E0F24E96E1050EF12FD
:1013E80001EE64F0D8901134E92613C0EEFF14C062
:1013F800EEFF1200116EEA6A860E1024E96E115093
:10140800EF1479E0080E1002F3500F24126E0C52FC
:1014180003E0020E0C6207D0D8901234640F166EE7
:101428000D50BFDE0BD00C4C03D0030E0C6206D05F
:10143800D8901234640F166E0D5001DF01EE64F07F
:10144800D8901234E926EECF14F0EECF15F00C50F8
:10145800020A07E0010A10E0030A2BE0010A34E05F
:1014680048D01450151008E1EA6A830E1024E96E7A
:101478001150EF12D8901200EA6AB10E1024E96EEA
:101488001150EF1436E1EA6A830E1024E96E115008
:10149800EF1A01EE64F0D8901234E92614C0EEFF7A
:1014A80015C0EEFFEA6AB10E1024E96E1150EF1272
:1014B80020D01450151008E1EA6A830E1024E96E52
:1014C8001150EF12D8901200EA6A830E1024E96EC8
:1014D8001150EF1201EE64F0D8901234E92614C0CE
:1014E800EEFF15C0EEFFEA6AB10E1024E96E115046
:1014F800EF12D88012000C50020A07E0010A05E03A
:10150800030A09E0010A07E013D0EA6AB10E1024C1
:10151800E96E111CEF16EA6AB10E1024E96E11503B
:10152800EF1406E1EA6A830E1024E96E111CEF1627
:10153800D8901200106E0F0E0D14116E0D38070B97
:10154800126E020A02E012662AD0080E0F02F35049
:101558000E24136E115207E0D8901334640F166EE0
:1015680011501FDE16D0020E126209D001EE64F08F
:10157800D8901334E9260A0EEE6EEF6A0AD0126686
:1015880008D001EE64F0D8901334E926010EEE6E0F
:10159800EF6AEA6AB10E0F24E96E1050EF121200DA
:1015A800236E2038030B256E269022BE26801F0E40
:1015B8002216000124B01DD0255005E0010A06E0DE
:1015C800030A0EE015D02286229A35D026A002D032
:1015D80023B01200229A228622A82DD022962BD040
:1015E8002234223221322298D8B02288228A23D06B
:1015F8001200255005E0010A09E0030A10E01AD09C
:101608002286100E20BC221A229A15D0229A100E79
:1016180020BC221A228622A80ED022960CD0223470
:10162800223221322298D8B02288228A080E20BC81
:10163800221A01D01200D89021362236D8902132B1
:101648003850E96E030E3924EA6E040EEF6E8ADA1A
:101658003850E96E030E3924EA6EB00E2510EF6E8D
:1016680081DA3850E96E030E3924EA6E21C0EFFFA3
:1016780079DA3850E96E030E3924EA6E22C0EFFF9A
:1016880071DA3650385C256E37503958266E26AEDA
:1016980002D0020E262626BE06D0E10E255C010EDB
:1016A8002658D8B027980A0EBB6F576A1200085000
:1016B8000914FF0AD8B4120026EE28F0010E0D6EA8
:1016C800030E0D602ED00F6A010E0E6E0E5227E02B
:1016D800DECF0AF0DFCF0BF00BBE19D0070E0B16CA
:1016E800DECF0CF0109031B810800C38030B0FE1EE
:1016F80008500A620CD009500B6209D0209010B033
:101708002080890E0D241E6E0E5040EC19F0060E36
:10171800D926000EDA220F2AD8900E36D7D70D2AEE
:10172800CFD71200176E1DB00ED020901DB22080AA
:10173800860E1E6E175040EC19F017508C130A0EC7
:10174800BB6F576AB4D01566B2D016B003D0171C59
:10175800B11704D0D8901730FF0AB11716B023D0AC
:1017680020801DB22090860E1E6E175040EC19F096
:1017780020801DB22090830E1E6E175040EC19F089
:1017880020901DB22080860E1E6ED890173440EC33
:1017980019F020901DB22080830E1E6ED890173449
:1017A80040EC19F07ED01DB21BD02090860E1E6E24
:1017B800175040EC19F02090830E1E6E175040EC25
:1017C80019F02090860E1E6ED890173040EC19F054
:1017D8002090830E1E6ED890173040EC19F061D01F
:1017E800D9CF1BF0DACF1CF0080E1602F3509B0F6E
:1017F800D96E090EDA6ADA220F0EDF14196E195043
:1018080006E0050A04E00F0A02E0050A23E1209039
:1018180019B22080860E1E6E175040EC19F02090E9
:1018280019B22080830E1E6E175040EC19F02090DC
:1018380019B02080860E1E6ED890173040EC19F033
:10184800209019B02080830E1E6ED890173040EC7F
:1018580019F023D02080860E1E6E175040EC19F028
:101868002080860E1E6ED890173040EC19F0080EB6
:10187800D95E000EDA5A5F0EDF140FE0060E16145A
:101888001A6E186E01EE64F0D8901834E926010E2D
:10189800EE6EEF6AD8901730B1131BC0D9FF1CC089
:1018A800DAFF835143EC11F00A0EBB6F576A12003E
:1018B800086E0F0E31140F6E30500E6E0D68010E4B
:1018C8000C6E0C52D8B410D10D2A080E0D02F3502C
:1018D800980FD96E090EDA6ADA220DA015D0080E13
:1018E800D95E000EDA5ADCCF09F0DD50149409BC39
:1018F8001484149609BE148614A602D014A404D025
:10190800080ED926000EDA22DECF10F0070EDF14FB
:10191800116EDECF09F0149409BC1484149609BE24
:101928001486DFCF0AF00938030B086238D00E504E
:10193800106235D00F50116232D0149231B814822F
:10194800020EDFBE141A08620BD008C015F01D90F5
:101958001D9214B21D820DC016F00C50E3DE1FD08C
:1019680014B411D014A60FD00DA00DD008C015F0D6
:101978001D9014B41D801D8214B21D920DC016F066
:101988000C50D0DE0CD008C015F01D9014B41D808A
:101998001D9214B21D820DC016F00C50C3DE030E4A
:1019A800D926000EDA22DFCF0BF0D8900A32D89071
:1019B8000A320BAE45D0030E0A1442E00B38030B73
:1019C80008623ED00F0EDD14136EDECF12F00E50FB
:1019D800126236D00F50136233D0149231B8148289
:1019E800020EDFBC141A030E0A14010A05E0030AEA
:1019F80006E0010A06E024D014B203D021D014B2C4
:101A08001FD014B411D014A60FD00DA00DD008C04B
:101A180015F01D9014B41D801D8214B21D920DC0C6
:101A280016F00C507FDE0CD008C015F01D9014B4D1
:101A38001D801D9214B21D820DC016F00C5072DE6E
:101A4800020ED926000EDA22DFCF0BF0D8900A3228
:101A5800D8900A320BAE45D0030E0A1442E00B3878
:101A6800030B08623ED00F0EDD14136EDECF12F0AA
:101A78000E50126236D00F50136233D0149231B820
:101A88001482020EDFBC141A030E0A14010A05E0C0
:101A9800030A06E0010A06E024D014B203D021D0DC
:101AA80014B21FD014B411D014A60FD00DA00DD0AD
:101AB80008C015F01D9014B41D801D8214B21D922B
:101AC8000DC016F00C502EDE0CD008C015F01D907D
:101AD80014B41D801D9214B21D820DC016F00C5056
:101AE80021DED8900C36EDD60E50120007A502D094
:101AF8003F6A4186120007A734D0070E0D14116EF5
:101B08000C50106EF80E105C030E11582AE3FC0EF0
:101B1800105C030E115825E2030E0C140F6ED890BA
:101B28000F360DB80F800F2C07D0EA6A8C0E0F24E1
:101B3800E96EEF68418415D0020E0F6208D0EA6A98
:101B48008C0E0F24E96E1F0EEF6E41840AD00F66CB
:101B580008D007A906D0EA6A8C0E0F24E96EEF6850
:101B680041841200382A000E3922386605D0020E48
:101B7800396202D0386A396A1200136A146A126A22
:101B8800100E126012D01350156E060E1424166E25
:101B98001350176EB50E1424186E98EC19F0400EF9
:101BA8001326000E1422122AEBD7136A146A14BEE5
:101BB80005D0E00E135C030E145811E213C01CF09C
:101BC80014C01DF01350E96E060E1424EA6EEE5090
:101BD8005BEC19F0132A000E14220001E8D715EC6B
:101BE8001AF02A82000159EC1AF02A920001120018
:101BF80007A31200342A342A02EE00F03450E926F2
:101C08007C0EEF6279D0342A02EE00F03450E926D7
:101C1800EFCF0CF0342A342A02EE00F03450E926D3
:101C2800EFCF09F0342A02EE00F03450E926D890BC
:101C3800EF34086E0934093208323F0E02150B6E74
:101C480003C60AF041B806D008500A6255D00950B8
:101C58000B6252D0342A342AFC0E0C14200A0BE0F2
:101C6800080A09E0040A1AE04C0A2BE0080A29E0ED
:101C78000C0A35E041D041A80CD007AF07D00CC002
:101C88000DF008C00EF009C00FF037D8010E9FDA2A
:101C980033D007AF31D07F0E9ADA2ED041B80CD0AE
:101CA8000CC00DF008C00EF009C00FF026D807AF21
:101CB80023D0010E8CDA20D007AF1ED07F0E87DA32
:101CC8001BD041A807D03ED9060107AF15D0400E5A
:101CD8007EDA12D007AF10D07F0E79DA0DD041B876
:101CE80007D030D9060107AF07D0400E70DA04D00C
:101CF80007AF02D07F0E6BDA120011EE20F00E0E45
:101D0800E66EE70EE66E0E0EE66E7C0EE66E0DC013
:101D1800E6FFE66AD8900E360F36D8900E320FC01E
:101D2800E6FF0EC0E6FFE66A166A02EE00F03450DF
:101D3800E926EFCF14F014C013F013380F0B136E0D
:101D4800342A02EE00F03450E926EFCF15F015C022
:101D580012F0129E14B0128E1790135051E1200EFB
:101D680012604ED0060E126202D0135205E0070E22
:101D780012620FD013660DD0060E125E000E135AB3
:101D88001250E96E060E1324EA6EEFCF16F0178094
:101D9800C4D0100E126202D0135205E0110E126266
:101DA8000FD013660DD00E0E125E000E135A12508D
:101DB800E96E060E1324EA6EEFCF16F01780ADD049
:101DC8001B0E126202D0135205E01C0E12620FD0D5
:101DD80013660DD0170E125E000E135A1250E96EDC
:101DE800060E1324EA6EEFCF16F0178096D01F0E5A
:101DF800126293D0136691D006C616F017808DD064
:101E0800135011E1400E12600ED0200E125E000E2B
:101E1800135A080E1224E96E060E1320EA6EEFCF4D
:101E280016F017807AD06F0E126206D0136604D0AF
:101E380007C616F0178071D0135003E1770E1264AD
:101E480012D0135010E112BE0ED0780E125E000EA2
:101E5800135AD80E1224E96E090E1320EA6EEFCF3A
:101E680016F017805AD0135002E112AE13D0135057
:101E780011E1F00E12600ED0800E125E000E135AA1
:101E8800280E1224E96E060E1320EA6EEFCF16F024
:101E9800178043D013521CE0020E136019D0066756
:101EA8000BD01306980E1224E96E060E1320EA6E64
:101EB800EFCF16F0178031D0062D2FD0980E1224B0
:101EC800E96E060E1320EA6EEFCF16F0178025D0C4
:101ED800010E13640FD0030E13600CD0020E135EB4
:101EE800980E1224E96E080E1320EA6EEFCF16F052
:101EF800178013D0020E136410D0400E125C030E2C
:101F080013580BE2030E135E980E1224E96E090EA5
:101F18001320EA6EEFCF16F01780149216BE1482C3
:101F280014C0E6FF15C0E6FF7F0E1614E66EE66ADB
:101F3800E66A17A004D00A0E0001BB6F576A418EEB
:101F480006011200119002EE00F03450E926EFCF9E
:101F580010F0342A02EE00F03450E926EFCF0FF0EB
:101F68000F9E10B00F8E342A02EE00F03450E9268E
:101F7800EFCF0DF00D9E10B20D8E10380F0B106EB6
:101F88001050000153E1200E0F6050D0060E0F6272
:101F980002D0105205E0070E0F620CD010660AD06E
:101FA800AA0E0D6203D1E9DDA10EBD6F0A0EBB6F4B
:101FB800576A1200100E0F6202D0105205E0110E7F
:101FC8000F6210D010660ED041A812000E0E0F5EE0
:101FD800000E105A0F50E96E060E1024EA6E0DC05E
:101FE800EFFFE4D01B0E0F6202D0105205E01C0E6A
:101FF8000F620ED010660CD0170E0F5E000E105A2E
:102008000F50E96E060E1024EA6E0DC0EFFFCED019
:102018001F0E0F62CBD01066C9D0060E0F6E106A65
:10202800E96E1024EA6E0DC0EFFFC0D0105014E125
:10203800400E0F6011D0200E0F5E000E105A080ED1
:102048000F24E96E060E1020EA6E0DC0EFFF080E91
:102058000F26000E1022AAD06F0E0F620ED0106647
:102068000CD0070E0F6E106AE96E060E1024EA6E89
:10207800020E0D10EF6E118099D0105003E1770E0B
:102088000F6419D0105017E10FBE15D0780E0F5EEF
:10209800000E105A3A0E0D6401D00D6ED80E0F24A2
:1020A800E96E090E1020EA6E0DC0EFFFD80E0F265C
:1020B800030E10227BD0105002E10FAE17D0105043
:1020C80015E1F00E0F6012D0800E0F5E000E105A50
:1020D800280E0F24E96E060E1020EA6E0DC0EFFFE1
:1020E800280E0F26000E1022118060D0105224E016
:1020F800020E106021D0060106670ED01006980E59
:102108000F24E96E060E1020EA6E0DC0EFFF980E40
:102118000F26000E10220ED0062D0CD0980E0F247C
:10212800E96E060E1020EA6E0DC0EFFF980E0F261E
:10213800000E102200013AD0010E10641ED0030ECA
:1021480010601BD0020E105E0F500E6E1050136EF2
:10215800030E126E13320E32122EFCD70E509ADA7C
:10216800980E0F24E96E080E1020EA6E0DC0EFFFDE
:10217800980E0F26020E102219D0020E106415D0E8
:10218800400E0F5C030E105810E2030E105E980EFE
:102198000F24E96E090E1020EA6E0DC0EFFF980EAD
:1021A8000F26030E1022118001D012000FC01CF060
:1021B80010C01DF00D505BEC19F0000111A003D008
:1021C80015EC1AF000010A0EBB6F576A12000D6E6B
:1021D8003850E96E030E3924EA6E040EEF6EC2DC45
:1021E8003850E96E030E3924EA6EB40EEF6EBADC8D
:1021F8003850E96E030E3924EA6E6F0EEF6EB2DCCA
:102208003850E96E030E3924EA6E0DC0EFFFAADCE0
:102218003650385C0E6E375039580F6E0FAE02D0FC
:10222800020E0F260FBE06D0E10E0E5C010E0F58EF
:10223800D8B027981200342A02EE00F03450E9266C
:102248006F0EEF6204D041AE02D0419E4C6A12007C
:10225800FA0E9312050E9412899881CF1CF01C90E7
:1022680082B01C801C9482B41C8489880001AF5100
:102278001C1A050E9316FA0E94161C5012001E6EA8
:10228800AE511E1A1EC081FF1EA082901EB0828011
:102298001EA482941EB482848B968B861200F950F9
:1022A8005344F92601D007D0800E4B6E7B6A200E6E
:1022B8007B60A5D0010C080E7B02F350980FE16EED
:1022C800080EE26AE2227B24D96E060EDA6ADA2266
:1022D800E6CF0CF00D6AE7CF0DF00E90DFBE0E8052
:1022E800070EDF14096E2AA43FD00EA03DD00CC003
:1022F8000FF00DC010F030C011F031C012F0000E18
:10230800DFEC16F014C008F0082C77D0070E0D1675
:102318000A680B6E0CC00FF00DC010F00AC011F067
:102328000BC012F091D8020E09620BD005EEC0F076
:102338007B50E9263C0EEF6E7BC00FF0090EA1D84A
:102348005ED0030E09620BD005EEC0F07B50E92683
:10235800140EEF6E7BC00FF0090E93D850D07BC0DF
:102368000FF0000E8ED84BD02AB447D00EB045D00F
:10237800070E0D14106E0C500F6E30C011F031C0E6
:1023880012F0000EDFEC16F014C008F0086602D058
:102398000DA604D0082C31D00DA62FD0F00E0D16A6
:1023A8000C6A0A6A0B6E0CC00FF00DC010F00AC060
:1023B80011F00BC012F048D8020E09620BD005EEDE
:1023C800C0F07B50E9263C0EEF6E7BC00FF0090E83
:1023D80058D815D0030E09620BD005EEC0F07B501B
:1023E800E926140EEF6E7BC00FF0090E4AD807D00D
:1023F8007BC00FF0000E45D802D07B2A58D7546A0C
:10240800800CF9505644F92601D005D07C6A200E7C
:102418007C6019D0010C05EEC0F07C50E926EF5025
:1024280010E005EEC0F07C50E926EF0605EEC0F09E
:10243800E926EF5006E17C502DD97CC00FF0080E3C
:1024480020D87C2AE4D7800C28EE98F0136A200E56
:10245800136016D0DECF14F0DDCF15F0125015162C
:102468001150141614500F6205D01550106202D086
:10247800135010D9080ED926000EDA22132AE7D7EE
:102488001200106E010E176E186A196A1A6A0F5038
:1024980008E01B6ED8901736183619361A361B2ED8
:1024A800F9D71A50A2131950A1131850A013175096
:1024B8009F131A50A6131950A5131850A413175098
:1024C800A313080E0F02F350980FE16E080EE26A8C
:1024D800E222E6CF15F0E5CF16F00FC011F0200E7E
:1024E8001160D4D01550E662CBD01650E762C8D040
:1024F800090E106204D0010E126EE65002D0040ECE
:10250800126EE650080E106204D0030E126201D05B
:102518007FD0010E126404D0E650E56201D078D075
:10252800E738D890E830070B146E040E146201D017
:102538006FD0176A186A196A1A6A1F0EE714136EA1
:10254800080E13600AD0010E176E13502CE01B6E94
:10255800D89017361B2EFCD726D0100E13600BD040
:10256800010E186E080E135C1EE01B6ED89018360C
:102578001B2EFCD718D0180E13600BD0010E196E45
:10258800100E135C10E01B6ED89019361B2EFCD76A
:102598000AD0010E1A6E180E135C05E01B6ED89057
:1025A8001A361B2EFCD71A50921319509113185033
:1025B800901317508F1314A408D01A50921B195057
:1025C800911B1850901B17508F1B030E1414010AEF
:1025D80005E0030A0CE0010A13E01AD01A5096131A
:1025E80019509513185094131750931311D01A506B
:1025F8009A1319509913185098131750971308D015
:102608001A509E1319509D1318509C1317509B1362
:10261800122E77D71050090A37E0080E1124E96EF8
:10262800060EEA6AEA22EF38D890E830030B010A6E
:1026380011E0030A05E0010A0DE0030A06E00AD0EA
:10264800030EE126000EE2221FD0030EE126000E43
:10265800E2221AD0E4CF00FA0A01016B0F0EE4144B
:10266800016F0189E7CF02FA02CA20F0248000CA6C
:1026780021F001CA22F0000ED4EC0AF0E65004D092
:10268800070EE126000EE222112A29D70A0EBB6F97
:10269800576A1200166E010E1C6E1D6A1E6A1F6AAA
:1026A800165008E0206ED8901C361D361E361F3690
:1026B800202EF9D71F1E1E1E1D1E1C1E1F50A217DE
:1026C8001E50A1171D50A0171C509F17080E160268
:1026D800F350980FE16E080EE26AE222E6CF1AF094
:1026E800E7CF1BF0040E176EE650010E176404D0F6
:1026F800E650E56201D072D0E738D890E830070B91
:10270800196E040E196201D069D01C6A1D6A1E6A0E
:102718001F6A1F0EE714186E080E18600AD0010E03
:102728001C6E18502CE0206ED8901C36202EFCD73A
:1027380026D0100E18600BD0010E1D6E080E185C06
:102748001EE0206ED8901D36202EFCD718D0180E0B
:1027580018600BD0010E1E6E100E185C10E0206E73
:10276800D8901E36202EFCD70AD0010E1F6E180EE8
:10277800185C05E0206ED8901F36202EFCD71F1E4F
:102788001E1E1D1E1C1E1F5092171E5091171D50F5
:1027980090171C508F17030E1914010A05E0030A3D
:1027A8000CE0010A13E01AD01F5096171E50951717
:1027B8001D5094171C50931711D01F509A171E5074
:1027C80099171D5098171C50971708D01F509E171F
:1027D8001E509D171D509C171C509B17172E84D7F1
:1027E800080E1624E96E060EEA6AEA22EF38D89037
:1027F800E830030B010A1AE0030A04E0010A02E0C8
:10280800030A14E0E4CF00FA0A01016B0F0EE41486
:10281800016F0189E7CF02FA02CA20F0248000CABA
:1028280021F001CA22F0000ED4EF0AF012007D2A2E
:10283800F00E7D6402D0010E7D6E7DC009F00A6A3B
:10284800280E0CEC01F0086E086608D09E51921B09
:102858009D51911B9C51901B9B518F1B7DC009F072
:102868000A6A3C0E0CEC01F0086E086609D09A5111
:10287800921B9951911B9851901B97518F1B11D006
:102888007DC009F00A6A500E0CEC01F0086E08666B
:1028980008D09651921B9551911B9451901B9351BE
:1028A8008F1B120026EE08F0086A200E08608AD0F6
:1028B800070EDE140B6E080E0802F3509A0F0C6E0A
:1028C800080E0D6A0D220CC0E1FF0DC0E2FF129246
:1028D8009FB11282D89012B2D880A233A133A0330C
:1028E8009F331294A3B11284D89012B4D880A6331F
:1028F800A533A433A33312B224D012A461D01F0E7F
:10290800E6140A6E01EED0F0E926EF501AE11F0E28
:10291800E6140A6E01EED0F0E926EF5012E11F0E20
:10292800E6140A6E01EED0F0E926EF500AE11F0E18
:10293800E7140A6E01EED0F0E926EF5002E1A69FF7
:102948003FD00CC0E9FF0DC0EAFF096A040E096018
:1029580037D01F0EEF140A6EEE38D890E830070B08
:10296800040A2CE08FC00EF090C00FF091C010F058
:1029780092C011F00A5008E0136ED890113210324C
:102988000F320E32132EF9D711EED0F00A50E1268D
:102998000B50010A02E0030A0CE10E321290D8B083
:1029A8001280E736E736E736D89012B0D880E73697
:1029B80005D00E3202E3E76801D0E76A092AC6D7D4
:1029C800082A73D712002F1C816E8B928B822B469C
:1029D8002BBA0AD0FD0E2B6ED8902C3602E1010ED0
:1029E8002C6E11EED0F00DD02BB403D011EED8F030
:1029F80008D02BB603D011EEE0F003D02BA811EECF
:102A0800E8F0086A080E096ED8802C50E614D8B48D
:102A1800D8900836092EF8D72F50081AD89008B839
:102A2800D880089808B60888089608B408860894D4
:102A380008B208840892D8B0088208C081FF08A0AC
:102A4800829008B0828008A4829408B482848B980B
:102A58008B882B18816E2BA482942BB482842FA48C
:102A680004D02BA482842BB482948B928B82120084
:102A78002B1E03E12E6A096A02D02DC009F0080E48
:102A8800086E8FC0A7F090C0A8F091C0A9F092C0BE
:102A9800AAF0070EA71507E0010A09E0030A0BE0F0
:102AA800060A0EE010D0099E2BBE098E0CD02B66AC
:102AB8000AD0099E08D02B6606D02E8E098E03D028
:102AC8002B6601D0098E09462B52D8B42E46030E28
:102AD8000A6ED890AA33A933A833A7330A2EF9D798
:102AE800082ED7D7F29C09C02DF0D8902DB8D880E1
:102AF8002D982DB62D882D962DB42D862D942DB27A
:102B08002D842D92D8B02D822DC081FF2DA08290CA
:102B18002DB082802DA482942DB482848B988B88CA
:102B28002BC081FF2BA482942BB482848B928B823E
:102B3800F28C2B6604D02E5202E0CC6ACA841200B2
:102B4800F9505444F92602D0BFD031D17A947E6A24
:102B5800400E7E602ED1080E7E02F350980FBF6F94
:102B6800060EC06BC023200E7E60C02BBFC0D9FFED
:102B7800C0C0DAFFDFAE1BD1040ED924E16E000E0F
:102B8800DA20E26E7A92E6CF09F0E7CF0AF00B6A14
:102B9800E7BC0B2ADFB802D0E7AE2DD0DFA802D001
:102BA8002AB404D0DFB82CD02AB42AD009C00FF038
:102BB8000AC010F030C011F031C012F00B50FBD831
:102BC80014C008F008BE1CD008B00DD001EE90F07B
:102BD8007E50E926EF9A08B0EF8A01EE90F0E926D8
:102BE800EF9008B0EF8001EE90F07E50E926EF906C
:102BF80008B0EF8005D001EE90F07E50E926EF8016
:102C0800060ED924E16E000EDA20E26EE6CF09F056
:102C1800E7CF0AF00B6AE7BC0B2ADFB602D0E7AEB3
:102C280028D0DFA602D02AB404D0DFB627D02AB431
:102C380025D009C00FF00AC010F030C011F031C023
:102C480012F00B50B8D814C008F008BE17D001EE27
:102C580090F07E50E926EFA004D001EE90F0E9262E
:102C6800EF8A01EE90F07E50E926EF9208B0EF82ED
:102C780005D001EE90F07E50E926EF820C90DFBC83
:102C88000C807AB406D07E50D3D87A92D8B07A82A3
:102C980006D001EE90F07E50E926EF98EF9601EE0F
:102CA80090F07E50E926EFB67A840CB07A947AA236
:102CB8007DD0D9CFE1FFDACFE2FFE4BE05D001EE47
:102CC80090F0E926EFB872D027A8010CBFC0D9FF51
:102CD800C0C0DAFFD9CFE1FFDACFE2FF070EE41474
:102CE8000FE0010A11E0030A13E0010A15E0070AE0
:102CF80017E0010A19E0030A1CE0010A1FE022D0CC
:102D0800010E086E096A1ED0050E086E096A1AD0EF
:102D18000A0E086E096A16D0320E086E096A12D0B9
:102D2800640E086E096A0ED0F40E086E010E096E64
:102D380009D0E80E086E030E096E04D0880E086EDE
:102D4800130E096EE738E8461F0B0F0B0A6E085082
:102D58000A02F3CF0BF0F4CF0CF00D6A09500A0207
:102D6800F3500C26F4500D220AAE04D008500C5E25
:102D780009500D5A09AE02D00A500D5E0B500C10C6
:102D88000D1012E005EE00F0030E7E02F350E92666
:102D98000BC0EEFF0CC0EEFF0DC0EEFF01EE90F091
:102DA8007E50E926EF8802D07E50EFD8020C7E2AAA
:102DB800CFD64B6A800C136E14682AA41AD0103828
:102DC800E8461F0B1F0B176E1238E8461F0B1F0B28
:102DD800186E070E101612160F50116227D01050D9
:102DE800126224D0146A1750186220D0010E146E93
:102DF8001DD01038030B176E1238E840E8423F0B1D
:102E0800030B186E1750186211D00F0E10161214FB
:102E1800166E1150156E0F50156208D010501662BC
:102E280005D0146A12B8142A1350141A1450120038
:102E38000D6E0F90080E0D02F350980FE16E060EFE
:102E4800E26AE222200E0D60E22A01EE90F00D50B7
:102E5800E926D890E73006E3EFB002D0EFA206D01B
:102E68000F8004D0EFA002D0EFB20F80D890E730E7
:102E7800030B0E6E0E5007E0010A1AE0030A2DE05C
:102E8800010A38E04FD00FA010D0EFB403D00FB034
:102E980003D006D00FB004D0EF86EF84D88012009C
:102EA800EFB640D0EF86D8801200EF96EF943AD074
:102EB8000FB010D0EFB403D00FB003D006D00FB0CE
:102EC80004D0EF86EF94D8801200EFB62BD0EF86AF
:102ED800D8801200EF96EF8425D0EFB403D00FB05E
:102EE80003D020D00FB01ED00FA0EF940FB0EF8406
:102EF800D88012000FA014D0EFBA02D0D8901200D8
:102F0800EFB403D00FB003D006D00FB004D0EF86D3
:102F1800EF84D8801200EFB605D0EF86D880120073
:102F2800EF96EF94D8901200F9505544F92602D044
:102F380006D024D07F6A400E7F6026D0010C01EEB7
:102F480090F07F50E926EFA81DD005EE00F0030EA3
:102F58007F02F350E926EE06000EEE5AEF5A05EE10
:102F680000F0030E7F02F350E926EE50EE10EF104A
:102F780009E101EE90F07F50E926EF9827A8020CAE
:102F88007F5003D87F2AD7D7800C0E6E080E0E020A
:102F9800F350980FE16E060EE26AE222200E0E60F0
:102FA800E22AE7AA0FD0020EE126000EE222E6CFBF
:102FB8000FF0106AE7CF10F00FC011F010C012F038
:102FC800CFD817D0020EE126000EE222E6CF0FF08E
:102FD800106A0F0EE714106E1088E7CF11F011C0B9
:102FE80020F024800FC021F010C022F0000ED4EF92
:102FF8000AF01200342A02EE00F03450E926EF50AD
:103008000B0A03E008680968FF0C342A02EE00F096
:103018003450E926EF507F0A03E008680968FF0C7E
:10302800342A02EE00F03450E926EF38070B030A81
:1030380003E008680968FF0C342A02EE00F03450F7
:10304800E926070EEF14010A03E008680968FF0C77
:10305800342A02EE00F03450E926EFCF08F008AC2D
:1030680003D008680968FF0CD8900836D89008364D
:10307800342A02EE00F03450E926EFCF09F0700E42
:10308800091AD8900932030E09140812093A094698
:103098001F0E0916342A02EE00F03450E926EFCF4D
:1030A8000AF00A3A0A42F80E0A160A50091208509B
:1030B800120002EE00F03450E926EFCF0AF0342A6D
:1030C80002EE00F03450E926D890EF34086E342A26
:1030D80002EE00F03450E9263F0EEF14096E0B9013
:1030E800EFBC0B80030E0A14020A05E0030A0DE088
:1030F800010A1EE033D00BB003D008680968FF0C42
:103108000890EFBA0880098E29D00BB00BD0EFBA1F
:1031180002D0EFA804D0EFAA05D0EFA803D0086822
:103128000968FF0CD890093208320996098C16D024
:103138000BA003D008680968FF0CD8900932083240
:1031480009B60BD008C00CF009C00DF006017FECE1
:103158000DF0086809680001FF0C09960850120074
:103168003850E96E030E3924EA6E0B0EEF6EB6EC9A
:103178000DF03850E96E030E3924EA6EED0EEF6E4D
:10318800B6EC0DF03850E96E030E3924EA6E0B0EDA
:10319800EF6EB6EC0DF03850E96E030E3924EA6E86
:1031A8007F0EEF6EB6EC0DF03850E96E030E392441
:1031B800EA6E310EEF6EB6EC0DF01238E8441F0BD4
:1031C800136E123A1242F80E1216030E111412124E
:1031D800D8901236700E121A1280129ED8901132A0
:1031E800D89011323850E96E030E3924EA6E010E78
:1031F800EF6EB6EC0DF03850E96E030E3924EA6E26
:1032080011C0EFFFB6EC0DF03850E96E030E39240B
:10321800EA6E12C0EFFFB6EC0DF03850E96E030EFF
:103228003924EA6E13C0EFFFB6EC0DF03850E96EA2
:10323800030E3924EA6EEF6AB6EC0DF03850E96EE9
:10324800030E3924EA6EEF6AB6EC0DF03650385C9E
:10325800136E37503958146E14AE02D0020E14266D
:1032680014BE06D0E10E135C010E1458D8B027988E
:103278000A0EBB6F576A12001F6E1EC0E9FFEA6A8A
:10328800D890EF14D8A4D88020A003D01F50EF12F4
:1032980002D01F1CEF161200A6B2FED71FC0A9FF4E
:1032A80020C0AAFFA69EA69CA680A85012001E6E4B
:1032B8001CC01FF01DC020F0EFDF1E18010132E016
:1032C800A6B2FED71EC0A8FF1CC0A9FF1DC0AAFF3A
:1032D800A69EA69CA684F29E550EA76EAA0EA76E61
:1032E800A682F28EA694622B000E6323E90E625D1D
:1032F800030E63590EE3626B636B602B000E612350
:10330800FE0E605D030E615904E3E00E606F030E6C
:10331800616F1CC01FF01DC020F0BEDF1E1802E048
:10332800D8901200D8801200A68EA69CF86A185071
:10333800F76EC00E1714F66E15C0E9FF16C0EAFF47
:10334800400E196E0900F552F5CFEEFF192EFAD787
:1033580012000BC0F6FF0CC0F7FFF86AA68EA69CF9
:103368000800F5501200010EC26E060EC16EBD0EA9
:10337800C06E070EB46E100E806EEF0E926E816AEC
:10338800050E936EC50E826EE00E946ED0A60AD01E
:10339800D0A408D000EE00F00F0EEE6AEA62FDD766
:1033A800E9AEFBD74A0EAF6EAC84AC98AB8EAB9847
:1033B800F26AF16AF06A9D6AA06A9F6AA26AD59E5B
:1033C800D66ACD6A480ECA6ECC6A630ECB6E9E92E0
:1033D8009D82B16A12000B6AB50E0C6EBADF0A6ED6
:1033E8001F6A206A59DF0A1809E00AC0A8FFA684E4
:1033F800550EA76EAA0EA76EA682A69406EE00F03A
:10340800086A096A08C01FF009C020F045DFEE6E9F
:10341800082A000E0922E00E085C030E0958F2E3A0
:103428001200156A0601030E156034D0EA6AAE0E62
:103438001524E96EEF6A156603D029EE98F007D0D7
:10344800152C03D026EE28F002D026EE68F0010EE7
:10345800166EDE50DE501552D8B4DE50176A080ECC
:10346800176016D0020E156203D0060E17600ED034
:10347800DFAE06D0EA6AAE0E1524E96E1650EF12DA
:10348800D8901636080ED926000EDA22172AE7D762
:10349800152AC9D707AB02D02F6801D02F6A07AD0C
:1034A80002D02A8601D02A961200FE0E1F6E030E45
:1034B800206EF2DE0101606F1F68030E206EECDEE5
:1034C800616F1B90FB0E605D030E615905E31B8065
:1034D800E00E606F030E616F2A90060107B12A8023
:1034E80001012AA015D02AA205D060C119F061C136
:1034F8001AF005D06029196E000E61211A6EFB0EB4
:10350800195C030E1A5804E3E00E196E030E1A6EC6
:10351800020E156E15BE3ED02AA02ED01BB002D0CA
:103528002AA202D0166A0AD0155060251F6E000E16
:1035380015BEFF0E6121206EAFDE166E15501924E0
:103548001C6E000E15BEFF0E1A201D6E1650AFDE43
:1035580015660CD0EA6A860E1524E96E16C0EFFFD0
:10356800EA6A8C0E1524E96EEF6806D0EA6A890EBD
:103578001524E96E16C0EFFF152C0AD02CEC11F0BB
:10358800166EEA6A860E1524E96E16C0EFFF010171
:103598001506C0D719C060F11AC061F1FE0E1C6E85
:1035A800030E1D6E605183DE1C68030E1D6E615193
:0235B8007ED6BD
:10B500000357EEE000E0001F000000000000000014
:10B51000000000000000000000000000000000002B
:10B5200000000000000000001020030000000000E8
:10B5300011200300000000001220030000000000A2
:10B54000132003000000000014200300000000008E
:10B55000152003000000000016200300000000007A
:10B56000172003000000000000200300000000007E
:10B570000120030000000000022003000000000082
:10B58000032003000000000004200300000000006E
:10B590000520030000000000000000000000000083
:10B5A000000000000000000000000000000000009B
:10B5B000000000000000000000000000000000008B
:10B5C000000000000000000000000000000000007B
:10B5D000000000000000000000000000000000006B
:10B5E000000000000000000000000000000000005B
:10B5F000000000000000000000000000000000004B
:10B60000000000000000000000000000000000003A
:10B61000000000000000000000000000000000002A
:10B62000000000000000000000000000000000001A
:10B63000000000000000000000000000000000000A
:10B6400000000000000000000000000000000000FA
:10B6500000000000000000000000000000000000EA
:10B6600000000000000000000000000000000000DA
:10B6700000000000000000000000000000000000CA
:10B6800000000000000000000000000000000000BA
:10B6900000000000000000000000000000000000AA
:10B6A000000000000000000000000000000000009A
:10B6B000000000000000000000000000000000008A
:10B6C000000000000000000000000000000000007A
:10B6D000000000000000000000000000000000006A
:10B6E000000000000000000000000000000000005A
:10B6F000000000000000000000000000000000004A
:10B700000000000000000000000000000000000039
:10B710000000000000000000000000000000000029
:10B720000000000000000000000000000000000019
:10B730000000000000000000000000000000000009
:10B7400000000000000000000000000000000000F9
:10B7500000000000000000000000000000000000E9
:10B7600000000000000000000000000000000000D9
:10B7700000000000000000000000000000000000C9
:10B7800000000000000000000000000000000000B9
:10B7900000000000000000000800008080800030F1
:10B7A0000900018181810030080802828282003014
:10B7B00009080383838300300A10048484840030E2
:10B7C0000B100585858500300A18068686860030B0
:10B7D0000B180787878700300C200888888800307E
:10B7E0000D200989898900300C280A8A8A8A00304C
:10B7F0000D280B8B8B8B00300E300C8C8C8C00301A
:10B800000F300D8D8D8D00300E380E8E8E8E0030E7
:10B810000F380F8F8F8F00301040109090900030B5
:10B820001140119191910030104812929292003083
:10B830001148139393930030125014949494003051
:10B84000135015959595003012581696969600301F
:10B8500013581797979700301460189898980030ED
:10B86000156019999999003014681A9A9A9A0030BB
:10B8700015681B9B9B9B003016701C9C9C9C003089
:10B8800017701D9D9D9D003016781E9E9E9E003057
:10B8900017781F9F9F9F00300000030000010002E7
:10B8A0000100030001010102020003000201020283
:10B8B0000300030003010302040003000401040267
:10B8C000050003000501050206000300060106024B
:10B8D00007000300070107022E2E2E2E2E2E2E2EDD
:020000040020DA
:080000000507000C00070003D6
:020000040030CA
:08000000FF021F08FF0181FF50
:00000001FF
